:100000000C942E000C94B00B0C944B000C944B00F1
:100010000C944B000C944B000C944B000C944B0034
:100020000C944B000C944B000C944B000C944B0024
:100030000C944B000C944B000C944B000C944B0014
:100040000C944B000C944B000C944B000C944B0004
:100050000C944B000C944B000C944B0011241FBECD
:10006000CFEFD8E0DEBFCDBF11E0A0E0B1E0E2E924
:10007000FCE102C005900D92AA3AB107D9F711E050
:10008000AAEAB1E001C01D92AA3FB107E1F70E94C0
:100090008E0D0C94470E0C940000FF920F931F934B
:1000A000CF93DF9309EC11E0CAE0D0E0FF24F39492
:1000B000CE010E94070E8150F8018E3F10F4F082AD
:1000C00001C0108221960F5F1F4FC431D10581F707
:1000D000C4E1D0E0CE010E94070E8F3F21F0FE0167
:1000E000EA50FF4F80832196CE31D10599F7CEE1BA
:1000F000D0E0CE010E94070E8F3F21F0FE01EF55A8
:10010000FE4F80832196C832D10599F7C8E2D0E02E
:10011000CE010E94070E8F3F21F0FE01E852FF4FF3
:1001200080832196C233D10599F7C2E3D0E0CE0196
:100130000E940F0E8F3FFFEF9F0729F0FE01E75847
:10014000FE4F918380832296C634D10581F7DF91DB
:10015000CF911F910F91FF900895999AA19A0895B8
:10016000999AA1980895813019F40D9A159A0895D5
:10017000823031F08330A1F0843029F40D9A159A41
:100180000C9A149A0895853049F0863019F40D9A26
:10019000159A06C0873031F40D9A159A0C9A149A64
:1001A0000B9A139A0895813019F40D9A15980895B1
:1001B000823031F08330A1F0843029F40D9A159803
:1001C0000C9A14980895853049F0863019F40D9AE8
:1001D000159806C0873031F40D9A15980C9A14982A
:1001E0000B9A139808951F93CF93DF93182FEB0169
:1001F0000E94B3002196D093ED01C093EC011093BF
:100200001701DF91CF911F9108950E94970C0E94D2
:100210009A0C80E40E947B0C8CE10E94820C8EE19F
:100220000E94820C8EE10E94820C8EE10E94820C60
:100230008EE10E94820C8EE10E94820C8EE10E946F
:10024000820C8CE10E94820C87E00E94820C8FE07D
:100250000E94820C8FE00E94820C8FE00E94820C30
:100260008FE00E94820C8FE00E94820C8FE00E943F
:10027000820C87E00E94820C8FE10E94820C8FE149
:100280000E94820C80E00E94820C80E00E94820C1E
:1002900080E00E94820C80E00E94820C8FE10E942C
:1002A000820C8FE10E94820C8EE10E94820C8CE114
:1002B0000E94820C80E00E94820C80E00E94820CEE
:1002C00080E00E94820C80E00E94820C88E10E9403
:1002D000820C8CE10E94820C8FE00E94820C87E0ED
:1002E0000E94820C80E00E94820C80E00E94820CBE
:1002F00080E00E94820C80E00E94820C83E00E94D9
:10030000820C87E00E94820C80E00E94820C80E0D8
:100310000E94820C80E00E94820C80E00E94820C8D
:1003200080E00E94820C80E00E94820C8FE10E949B
:10033000820C8FE10E94820C80E00E94820C80E09F
:100340000E94820C80E00E94820C80E00E94820C5D
:1003500080E00E94820C80E00E94820C87E00E9474
:10036000820C8FE00E94820C8FE10E94820C8FE150
:100370000E94820C80E00E94820C80E00E94820C2D
:1003800080E00E94820C80E00E94820C80E00E944B
:10039000820C80E00C94820C80E40E947B0C84E050
:1003A0000E94820C84E00E94820C8AE00E94820CEF
:1003B0008AE00E94820C81E10E94820C81E10E940D
:1003C000820C81E10E94820C8EE00E94820C84E00B
:1003D0000E94820C84E00E94820C84E00E94820CC5
:1003E00084E00E94820C8AE00E94820C81E10E94DB
:1003F000820C8FE10E94820C80E00E94820C8AE0D5
:100400000E94820C84E00E94820C8EE00E94820C8A
:1004100080E10E94820C80E10E94820C81E10E94B6
:10042000820C8EE00E94820C80E00E94820C84E0AC
:100430000E94820C84E00E94820C8EE00E94820C5A
:100440008FE10E94820C80E00E94820C85E10E9474
:10045000820C80E00E94820C8AE00E94820C85E17E
:100460000E94820C80E00E94820C8AE00E94820C32
:1004700080E00E94820C85E10E94820C80E00E9454
:10048000820C8AE00E94820C80E00E94820C84E050
:100490000E94820C84E00E94820C84E00E94820C04
:1004A00084E00E94820C8EE00E94820C8FE10E9408
:1004B000820C80E00E94820C8AE00C94820C611510
:1004C000710511F4806804C06130710519F4806C05
:1004D0000C947B0C0895CF93C82F80680E947B0CEE
:1004E00081E00E94820C87E00E94820C80E00E94E2
:1004F000820C8C2F806C0E947B0C81E00E94820C0D
:1005000085E00E94820C80E0CF910C94820CCF9306
:10051000C82F80680E947B0C80E20E94820C80E2DF
:100520000E94820C80E00E94820C8C2F806C0E94C2
:100530007B0C80E20E94820C80E20E94820C80E0B0
:10054000CF910C94820CCF93C82F80680E947B0CB3
:1005500084E00E94820C82E00E94820C80E00E9473
:10056000820C8C2F806C0E947B0C81E00E94820C9C
:1005700085E00E94820C85E0CF910C94820CCF9391
:10058000C82F80680E947B0C84E00E94820C82E06D
:100590000E94820C80E00E94820C8C2F806C0E9452
:1005A0007B0C86E00E94820C85E00E94820C80E039
:1005B000CF910C94820CCF93C82F80680E947B0C43
:1005C00081E00E94820C85E00E94820C80E00E9403
:1005D000820C8C2F806C0E947B0C80E20E94820C2B
:1005E00080E20E94820C80E0CF910C94820CCF9329
:1005F000C82F80680E947B0C81E00E94820C82E000
:100600000E94820C83E00E94820C8C2F806C0E94DE
:100610007B0C86E00E94820C85E00E94820C80E0C8
:10062000CF910C94820CCF93C82F80680E947B0CD2
:1006300081E00E94820C82E00E94820C83E00E9492
:10064000820C8C2F806C0E947B0C81E00E94820CBB
:1006500085E00E94820C80E0CF910C94820CCF93B5
:10066000C82F80680E947B0C81E00E94820C87E08A
:100670000E94820C80E00E94820C8C2F806C0E9471
:100680007B0C80E20E94820C80E20E94820C80E05F
:10069000CF910C94820CCF93C82F80680E947B0C62
:1006A00081E00E94820C82E00E94820C80E00E9425
:1006B000820C8C2F806C0E947B0C81E00E94820C4B
:1006C00085E00E94820C80E0CF910C94820CCF9345
:1006D000C82F80680E947B0C81E00E94820C82E01F
:1006E0000E94820C80E00E94820C8C2F806C0E9401
:1006F0007B0C86E00E94820C85E00E94820C80E0E8
:10070000CF910C94820CCF93C82F80680E947B0CF1
:1007100081E00E94820C80E00E94820C8C2F806C11
:100720000E947B0C81E00E94820C80E0CF910C94AF
:10073000820C0F931F93CF93DF93EC018B010097F3
:1007400021F4CB010E946B021CC08130910521F481
:10075000CB010E94870215C08230910521F4CB01A4
:100760000E94A30215C08330910521F4CB010E94A1
:10077000BF0222C08430910521F4CB010E94DB022C
:1007800025C0C530D10521F4C8010E94F70228C058
:10079000C630D10539F4C801DF91CF911F910F9177
:1007A0000C941303C730D10539F4C801DF91CF9100
:1007B0001F910F910C942F03C830D10539F4C80153
:1007C000DF91CF911F910F910C944B03C930D1054C
:1007D00039F4C801DF91CF911F910F910C946703F9
:1007E0002C9739F4C801DF91CF911F910F910C9490
:1007F0008303DF91CF911F910F9108958091F001B4
:1008000060E070E090E00E9499038091F10163E064
:1008100070E090E00E94990387E090E00E948303DB
:100820008091F2016AE070E090E00E94990380916B
:10083000F3016DE070E090E00C949903FF920F9348
:100840001F93CF93DF93CDB7DEB760970FB6F894C1
:10085000DEBF0FBECDBFF82E062F142F89E08F15F7
:1008600020F08BE191E00E94A90C4AE050E0BE012B
:100870006F5F7F4F8F2D90E00E94E60DCE010196B5
:100880000E94A90C8DE191E00E94A90C0A3020F48D
:100890008BE191E00E94A90C4AE050E0BE016F5F3D
:1008A0007F4F802F90E00E94E60DCE0101960E94BE
:1008B000A90C8DE191E00E94A90C1A3020F48BE183
:1008C00091E00E94A90C4AE050E0BE016F5F7F4FAB
:1008D000812F90E00E94E60DCE0101960E94A90CA6
:1008E00060960FB6F894DEBF0FBECDBFDF91CF91FB
:1008F0001F910F91FF9008950F931F93CF93DF9354
:10090000CDB7DEB760970FB6F894DEBF0FBECDBF90
:10091000082F162F8A3020F48BE191E00E94A90C59
:100920004AE050E0BE016F5F7F4F802F90E00E9451
:10093000E60DCE0101960E94A90C8DE191E00E9486
:10094000A90C1A3020F48BE191E00E94A90C4AE036
:1009500050E0BE016F5F7F4F812F90E00E94E60D57
:10096000CE0101960E94A90C60960FB6F894DEBFE6
:100970000FBECDBFDF91CF911F910F9108959CE3E2
:10098000699FB0011124640F711D20E13EE0482FE2
:10099000429FC001439F900D1124860F971F089519
:1009A0009C0160E17EE00E94D20D6093E4016091C1
:1009B000E40140EF51EF649FC001659F900D112449
:1009C000820F931F6CE370E00E94D20D6093E301ED
:1009D0003091E3019091E40184EC389F802D112443
:1009E00040EF949F800D1124820F8093E2010895BF
:1009F000982F92959F708F702AE0929F800D1124FE
:100A000008956AE00E94C60D20E1829F900D112496
:100A1000892F08951F93CF93DF931F92CDB7DEB731
:100A2000182F69830E94FA0C0E94030D82EA0E942B
:100A30001E0D812F0E941E0D6981862F0E940105C7
:100A40000E941E0D0F90DF91CF911F910C940E0DFF
:100A50001F93CF93DF931F92CDB7DEB7182F0E945D
:100A6000FA0C0E94030D82EA0E941E0D812F0E9443
:100A70001E0D0E940E0D0E94030D83EA0E941E0DA2
:100A800080E00E94530D89830E940E0D89810F9092
:100A9000DF91CF911F910895CF93DF938091F4015F
:100AA0006091F5019091F201D091F3012AE0929FBB
:100AB000D00D11249091F001C091F1012AE0929F94
:100AC000C00D11249AE0899F600D112482E00E94DC
:100AD0000A056D2F83E00E940A056C2F84E0DF91E8
:100AE000CF910C940A05CF93DF9384E00E942805F0
:100AF000D82F83E00E942805C82F82E00E94280595
:100B00009D2F9073969596959695292F220F220FDB
:100B1000290FDF702D0F9C2F9077969596959695BF
:100B2000392F330F330F390FCF703C0F482F4077D9
:100B3000469546954695942F990F990F940F8F706F
:100B4000980F4AE0892F642F0E94C60D8093F4010C
:100B50009093F501832F0E94C60D8093F20190932C
:100B6000F301822F0E94C60D8093F0019093F10152
:100B7000DF91CF91089580E480937C0087E8809393
:100B80007A00089580917C0080937C0080917A00A7
:100B9000806480937A0080917A0084FFFCCF8091FA
:100BA0007A00806180937A0080917800909179003A
:100BB0009093F9018093F801089580917C00816001
:100BC00080937C0080917A00806480937A00809189
:100BD0007A0084FFFCCF80917A00806180937A0054
:100BE00080917800909179009093F7018093F601BD
:100BF000089580917C0080937C0080917A008064CD
:100C000080937A0080917A0084FFFCCF80917A00F3
:100C1000806180937A008091780090917900909320
:100C2000F9018093F80180917C00816080937C00C1
:100C300080917A00806480937A0080917A0084FFAA
:100C4000FCCF80917A00806180937A008091780057
:100C5000909179009093F7018093F6010895CF93D6
:100C6000C82F862F642F0E94890CC13019F48FE1A0
:100C700091E01DC0C23019F483E291E018C0C33086
:100C800019F487E291E013C0C43019F48BE291E0CB
:100C90000EC0C53019F48FE291E009C0C63019F4D6
:100CA00083E391E004C0C73029F487E391E0CF915A
:100CB0000C94A90CCF9108958CE00E94C40C51981B
:100CC000599AE89AE9E6F0E080818260808378941E
:100CD0000E94BB050E94FA0C0E94030D82EA0E944A
:100CE0001E0D8DE00E941E0D83E80E941E0D0E94C5
:100CF0000E0D57985F9A56985E9A55985D9A54983B
:100D00005C9A0E94AD000E9473050C944D004F99AF
:100D100019C02FE788E391E0215080409040E1F72F
:100D200000C000004F9B02C081E008954F99FCCFA6
:100D30002FEF89EF90E0215080409040E1F700C014
:100D40000000F4CF80E008954E9910C02FE788E3AB
:100D500091E0215080409040E1F700C0000089B14F
:100D600086FB882780F991E08927089580E008951F
:100D70004D9921C02FE788E391E0215080409040B9
:100D8000E1F700C000004D9B02C081E00895809112
:100D9000EE01823021F08091EE018330B1F74D9960
:100DA000F4CF2FEF89EF90E0215080409040E1F7A1
:100DB00000C00000F4CF80E008951092AA012091B5
:100DC000E9016091EA019091EB01809119013CE306
:100DD000639FB0011124620F711D40E15EE0949F9A
:100DE0009001959F300D1124620F731F0C94F30036
:100DF0004C9935C02FE788E391E021508040904026
:100E0000E1F700C000004C9B07C08091AA0183332A
:100E1000C0F00E94DD0623C08091EE018230A9F768
:100E20004C99F3CF2FEF89EF90E021508040904014
:100E3000E1F700C000008091AA018F5F8093AA01B2
:100E4000EFCF4C990AC02FEF89EF90E021508040FE
:100E50009040E1F700C00000F4CF81E0089580E009
:100E600008951F93CF93DF938091EE01811124C0E9
:100E70008091F1018F5F8093F1018091F1018A30BF
:100E800038F01092F1018091F0018F5F8093F001B2
:100E90008091F001823040F08091F101843020F0A7
:100EA0001092F1011092F0011092F5011092F401EC
:100EB0000E94FE030E944C058091EE01813021F4D6
:100EC000809119010E94B3008091EE01823069F592
:100ED0008091E80181110BC08091EB018F5F8093BD
:100EE000EB018091EB01883110F01092EB018091C1
:100EF000E801813059F48091EA018F5F8093EA0123
:100F00008091EA018C3310F01092EA018091E8019F
:100F1000823059F48091E9018F5F8093E9018091DB
:100F2000E9018C3310F01092E9018091EE018330D9
:100F300009F0EEC08091D30181110CC08091E401D1
:100F40008F5F8093E4018091E401883128F0109252
:100F5000E40102C080E001C081E09091D3019130B2
:100F600061F48091E3018F5F8093E3018091E3015D
:100F70008C3310F01092E30181E09091D301923014
:100F800061F48091E2018F5F8093E2018091E20140
:100F90008C3310F01092E20181E09091D3019330F4
:100FA00061F4909116019F5F909316019091160144
:100FB000983128F01092160102C0D0E001C0D1E0B3
:100FC0009091D301943061F49091DC019F5F9093F4
:100FD000DC019091DC019C3310F01092DC01D1E037
:100FE0009091D301953069F4909115019F5F909392
:100FF000150190911501983030F091E09093150112
:1010000002C010E001C011E09091D301963061F46C
:101010009091DB019F5F9093DB019091DB01923017
:1010200028F01092DB0102C0C0E001C0C1E08823BB
:1010300031F18091E2016091E3014091E4019CE390
:10104000699FB0011124680F711D20E13EE0429FAD
:10105000C001439F900D1124680F791FE091DD01BD
:10106000F0E0EE0FFF1FE555FE4F71836083809126
:10107000DD0190E04996880F991F0E94220EDD2322
:1010800001F1E091DD0180911601F0E0E65FFE4F95
:101090008083E091DD018091DC01F0E0E154FE4FBE
:1010A0008083609116018091DD0190E044960E945A
:1010B000150E6091DC018091DD0190E04E960E945A
:1010C000150E112381F0E091DD0180911501F0E012
:1010D000E050FF4F8083609115018091DD0190E029
:1010E00088960E94150ECC2399F0E091DD01809145
:1010F000DB01F0E0E753FE4F80836091DB018091DC
:10110000DD0190E00A96DF91CF911F910C94150EAE
:10111000DF91CF911F9108958091EE0181111EC042
:101120008091F3018F5F8093F3018091F3018A3006
:1011300038F01092F3018091F2018F5F8093F201F9
:101140008091F201863010F01092F2011092F501B8
:101150001092F4010E94FE030E944C058091EE0162
:10116000813021F4809119010E94D3008091EE0119
:10117000823059F48091E8018F5F8093E80180917B
:10118000E801833010F01092E8018091EE01833085
:1011900059F48091D3018F5F8093D3018091D30163
:1011A000873010F01092D30108950F931F93CF93BF
:1011B000DF93CDB7DEB760970FB6F894DEBF0FBEF2
:1011C000CDBF082F162F8A3020F48BE191E00E94CA
:1011D000A90C4AE050E0BE016F5F7F4F802F90E086
:1011E0000E94E60DCE0101960E94A90C8DE191E0CE
:1011F0000E94A90C1A3020F48BE191E00E94A90C06
:101200004AE050E0BE016F5F7F4F812F90E00E9467
:10121000E60DCE0101960E94A90C60960FB6F894D7
:10122000DEBF0FBECDBFDF91CF911F910F9108950B
:10123000882321F00E9405010C94FE030895882361
:1012400069F00E94970C0E949A0C8BE391E00E9437
:10125000A90C40E06CE081E00E942F0690911901FA
:1012600080911801981751F08091190140E06CE0CD
:101270000E942F06809119018093180108958823F8
:1012800069F10E94970C0E949A0C89E491E00E94F7
:10129000A90C61E080E00E94890C87E591E00E9442
:1012A000A90C1092EB011092EA011092E901109240
:1012B000E80161E087E00E94890C4091E9016091BA
:1012C000EA018091EB010E941E0481E080931901E4
:1012D0008091190140E06CE00E942F069091190165
:1012E00080911801981751F08091190140E06CE04D
:1012F0000E942F0680911901809318019091E701B7
:101300008091EB0198130CC09091E6018091EA0165
:10131000981306C09091E5018091E901981731F189
:1013200061E087E00E94890C8FE591E00E94A90CA2
:1013300061E087E00E94890C4091E9016091EA0137
:101340008091EB010E941E048091190140E06CE045
:101350000E942F068091EB018093E7018091EA01C2
:101360008093E6018091E9018093E5010895CF9390
:10137000DF93CDB7DEB760970FB6F894DEBF0FBE30
:10138000CDBF882309F4ACC00E94970C0E949A0C30
:101390000E94CC0180EC0E947B0C80E00E94820CB9
:1013A00080E80E947B0C81E00E94820C8FEC0E94FE
:1013B0007B0C84E00E94820C8FE80E947B0C85E00D
:1013C0000E94820C82E80E947B0C82E00E94820CC8
:1013D00060E083E00E94890C8BE691E00E94A90CFA
:1013E0008091DD0190E04AE050E0BE016F5F7F4FE9
:1013F00001960E94E60DCE0101960E94A90C89E695
:1014000091E00E94A90CE091DD01F0E0EE0FFF1FDA
:10141000E555FE4F808191810E94D0048091DD01CD
:1014200060E0893010F486E001C087E00E94890CFA
:101430004091E2016091E3018091E4010E941E0469
:1014400061E082E00E94890CA091DD01E091DD0164
:10145000B0E0A154BE4FF0E0E65FFE4F6C9180819A
:101460000E947C0489E691E00E94A90CE091DD01D4
:10147000F0E0E050FF4F41E068E080810E942F06DD
:10148000E091DD01F0E0E753FE4F8081882319F001
:101490008DE691E002C082E791E00E94A90CE09104
:1014A000DD01F0E0E65FFE4F808180931601E09160
:1014B000DD01F0E0E154FE4F80818093DC01E0919A
:1014C000DD01F0E0E050FF4F808180931501E09155
:1014D000DD01F0E0E753FE4F80818093DB019CC08B
:1014E0009091E4018091D90198130CC09091E3018F
:1014F0008091D801981306C09091E2018091D701A4
:101500009817F1F08091DD0160E0893010F486E0F9
:1015100001C087E00E94890C4091E2016091E301E3
:101520008091E4010E941E048091E4018093D9011E
:101530008091E3018093D8018091E2018093D701EB
:101540009091160180911401981306C09091DC01CE
:101550008091D601981791F061E082E00E94890C99
:101560006091DC01809116010E947C048091DC0175
:101570008093D601809116018093140190911501FA
:101580008091D501981771F0E091DD01F0E0E05015
:10159000FF4F41E068E080810E942F068091150195
:1015A0008093D5019091DB018091D401981799F037
:1015B00061E08BE00E94890C8091DB01882319F0A7
:1015C0008DE691E002C082E791E00E94A90C809133
:1015D000DB018093D4019091DD018091DA019817AD
:1015E000D9F060E084E00E94890C8091DD0190E0F8
:1015F0004AE050E0BE016F5F7F4F01960E94E60D0A
:10160000CE0101960E94A90C89E691E00E94A90CE6
:101610008091DD018093DA0160960FB6F894DEBF09
:101620000FBECDBFDF91CF9108958091EE01813043
:1016300021F08091EE01823069F4809119018F5F71
:1016400080931901809119018830E0F181E0809345
:10165000190108958091EE01833081F58091DD01BB
:101660008F5F8093DD018091DD018A3010F0109250
:10167000DD01E091DD01F0E0E65FFE4F80818093C7
:101680001601E091DD01F0E0E154FE4F808180938E
:10169000DC01E091DD01F0E0E050FF4F80818093BC
:1016A0001501E091DD01F0E0E753FE4F808180936A
:1016B000DB011092D30181E00C94B70984B392E06E
:1016C000892784BB08950E948706882361F0809152
:1016D000EE01853019F41092EE0105C08091EE0103
:1016E0008F5F8093EE010E94A40681110E94310752
:1016F0000E94B80681110E948C080E94F806811190
:101700000C94150B0895089508952091EE01909181
:101710001A0181E0291301C080E09091EE019093BD
:101720001A019091EE01911102C00C941809909148
:10173000EE01913011F40C941F099091EE0192305A
:1017400011F40C943F099091EE01933011F40C9434
:10175000B7098091EE01843011F08091EE01089577
:101760001F920F920FB60F9211242F933F934F9316
:101770005F936F937F938F939F93AF93BF93EF93F9
:10178000FF938091F5018F5F8093F5018091F501C2
:101790008A3038F01092F5018091F4018F5F8093C8
:1017A000F4018091F401863050F01092F4018091A0
:1017B000F3018F5F8093F30181E08093EF018091CB
:1017C000F3018A3038F01092F3018091F2018F5FBB
:1017D0008093F2018091F201863038F01092F2018C
:1017E0008091F1018F5F8093F1018091F1018A3046
:1017F00038F01092F1018091F0018F5F8093F00139
:101800008091F001823040F08091F101843020F02D
:101810001092F1011092F0018091EF01882341F0C4
:101820008091EE01811104C01092EF010E94FE032D
:10183000809117018930B1F08091EC019091ED0118
:1018400001979093ED018093EC018091EC019091D0
:10185000ED01892B39F4809117010E94D30089E0B2
:1018600080931701FF91EF91BF91AF919F918F915D
:101870007F916F915F914F913F912F910F900FBE8C
:101880000F901F901895449A00C044980895CF93E4
:10189000DF931F92CDB7DEB7662311F0459A01C0E2
:1018A00045983B9A3A9A399A389A40984198429882
:1018B000439887FD409A86FD419A85FD429A84FDB2
:1018C000439A89830E94430C4098419842984398D8
:1018D000898183FD409A82FD419A81FD429A80FD73
:1018E000439A0E94430C439A429A419A409A0F901D
:1018F000DF91CF910895E0EAFFE03197F1F760E0E2
:101900000C94470CE0EAFFE03197F1F761E00C94AA
:10191000470C611102C0805801C080540C947B0CAC
:1019200080EA9FE00197F1F781E090E0089581E07F
:101930000C947B0C82E00C947B0CE0EAFFE0319786
:10194000F1F78A3019F480EC0C947B0C61E00C9474
:10195000470CCF93DF93EC018991882319F00E9403
:101960009D0CFACFDF91CF910895CF93DF93FC01C7
:101970008491EF012196882321F00E949D0CFE01A5
:10198000F7CFDF91CF910895CF93C82F3D9A3C9A1E
:101990003B9A3A9A399A389AE0E0FAEF3197F1F7A0
:1019A000429A439A0E94430CE0E0FEE43197F1F73B
:1019B0000E94430CE0E0F1E03197F1F70E94430C04
:1019C000E0E0F1E03197F1F743980E94430CE0E04A
:1019D000F1E03197F1F788E20E947B0C88E00E94E9
:1019E0007B0C0E94970C86E00E947B0C8C2FCF9181
:1019F0000C947B0C8EB180728EB98EB180718EB9D1
:101A00006D986C9808956C9880E590E00197F1F7D7
:101A10006D9A80E590E00197F1F708956D9A80E561
:101A200090E00197F1F76C9880E390E00197F1F76F
:101A30006D9880E590E00197F1F7089598E040E314
:101A400050E020E530E06C9AFA013197F1F787FF1A
:101A500002C06D9801C06D9AF9013197F1F76C9849
:101A6000F9013197F1F7649BFECF880F915059F738
:101A70006C9A80E390E00197F1F76D9880E590E033
:101A80000197F1F76C9880E590E00197F1F78CB140
:101A90006C9AE0E5F0E03197F1F785FB882780F953
:101AA00091E089270895982F20E030E080E040E51C
:101AB00050E060E870E06C9AFA013197F1F76C98A9
:101AC000FA013197F1F7649BFECF659B08C0FB01DB
:101AD000022E02C0F595E7950A94E2F78E2B2F5F50
:101AE0003F4F2830310539F76C9AE0E3F0E0319749
:101AF000F1F7992311F06D9A01C06D98E0E5F0E0DF
:101B00003197F1F76C98E0E5F0E03197F1F76C9AD6
:101B1000E0E5F0E03197F1F76D9808950E945C06DA
:101B200087E791E00E94A90C2FEF83E294EF215008
:101B300080409040E1F700C000000E94970C0E9496
:101B40009A0C82E991E00E94A90C2FEF8BE792E9B1
:101B5000215080409040E1F700C000000E94970CA7
:101B60000E949A0C0E94B0000E9405010E94FE0390
:101B70000E94630B0E94850B2FEF81EE94E02150B1
:101B800080409040E1F700C00000F2CF991B79E05F
:101B900004C0991F961708F0961B881F7A95C9F7FD
:101BA00080950895AA1BBB1B51E107C0AA1FBB1F4C
:101BB000A617B70710F0A61BB70B881F991F5A95D9
:101BC000A9F780959095BC01CD010895FB019F0177
:101BD000E8944230C4F04532B4F44A3029F497FB1B
:101BE0001EF4909581959F4F642F77270E94D20D08
:101BF000805D8A330CF0895D8193CB010097A1F75A
:101C000016F45DE251931082C9010C94270EF999E4
:101C1000FECF92BD81BDF89A992780B50895A8E1BD
:101C2000B0E042E050E00C94390E262FF999FECF37
:101C300092BD81BD20BD0FB6F894FA9AF99A0FBEF5
:101C4000019608950E94150E272F0C94160EDC01A4
:101C5000FC01672F71917723E1F7329704C07C91E3
:101C60006D9370836291AE17BF07C8F30895DC01CE
:101C7000CB01FC01F999FECF06C0F2BDE1BDF89A97
:101C8000319600B40D9241505040B8F70895F89441
:021C9000FFCF84
:101C9200070707070707070707070C0C0C0C0C0CB4
:101CA2000C0C0C0C0C070C0901010930003A006104
:101CB200202000206220002020630061622000209A
:101CC2006263006120630061626300546573742083
:101CD2006F6B727568753A20005A61706E69206F79
:101CE2006B7275683A20006E612063617320002078
:101CF20020202020202020202020002E00205A41B9
:101D0200500020565950004E697472616D3134375B
:101D12000A506F6C696576616E696574657261738C
:101D220079005665727A69612076310A56656C6B64
:0A1D32006520686F64696E79000097
:00000001FF
